:1000000061288F00220884002009282084138F088B
:1000100003195C28F03091000E0880389000F03011
:1000200091030319910003198F0303195C28182801
:100030002B2003010C1820088E1F20088E0803199E
:100040000301900F252880060C28262800000F2881
:10005000841780055C280D080C0403198C0A803075
:100060000C1A8D060C198D068C188D060D0D8C0D35
:100070008D0D5C288F018E00FF308E07031C8F07CB
:10008000031C5C2803308D00DF3048203C288D01A4
:10009000E83E8C008D09FC30031C51288C070318A6
:1000A0004E288C0764008D0F4E280C1857288C1C86
:1000B0005B2800005B28080083130313831264008D
:1000C0000800831603308500013086000530831256
:1000D000A2000830A00073308E000A3001203230B8
:1000E0008E000A3001206400051C80280530A20023
:1000F0000830A00064308E000A30012014303A200D
:100100006400851C97280530A2000830A0005030FC
:100110008E001430012028303A200530A20008302B
:10012000A0006E308E001430012028303A20732851
:0401300063009828A8
:02400E00F53F7C
:00000001FF
